:1000000013EF25F0FFFFFFFF4CC05CF14BC05BF12D
:10001000E9CF01F1EACF02F1E1CF03F1E2CF04F140
:100020009E6A2C0ECE6ECF0ECF6E4C6A89B84C2ACB
:10003000010E4C184B6E000E4BB0100E8918100BB1
:10004000891A30EC00F001C1E9FF02C1EAFF03C1E7
:10005000E1FF04C1E2FF5CC14CF05BC14BF0110059
:10006000014A022A800E02184B6E800E4B5C02E1A0
:100070000A0E015C2CE3016A026A050E0012034AB3
:10008000042A800E04184B6E800E4B5C02E13C0E7D
:10009000035C1DE3036A046A0082054A062A800E97
:1000A00006184B6E800E4B5C02E13C0E055C0FE3C4
:1000B000056A066A074A082A800E08184B6E800EE9
:1000C0004B5C02E1180E075C02E3076A086A120043
:1000D0000001568456AE74EF00F0010E4E6E4D6A6C
:1000E0004C6A4B6A55364D32FF0E1200000155AE78
:1000F0004D9E000E12000001568256AE86EF00F0B3
:100100004E684D684C684B6855364D32FF0E1200F4
:1001100000014D6A4C6A4B6A536A4E6A000E120027
:10012000000157B0D3EF00F057A27BEF01F0596AFE
:10013000000E4D64EAEF00F0F00E4D14D8A4B5EFB8
:1001400000F04D3A4C380F0B4D264C38F00B4C6EEE
:100150004B380F0B4C264B38F00B4B6E53380F0BB4
:100160004B265338F00B536E5984D8904DBECEEFCA
:1001700000F053364B364C364D36592A4DBECEEF35
:1001800000F053364B364C364D36592A4DBECEEF25
:1001900000F053364B364C364D36592A59504E6482
:1001A0006FEF01F04E5E56BC53AE75EF01F0D88094
:1001B000800E53644B30000E4B224C224D22D8A0AF
:1001C00075EF01F04D324C324B324E4A7BEF01F06D
:1001D00075EF01F04CC04DF04BC04CF053C04BF0EC
:1001E000536A000E59864D6421EF01F0F00E4D1454
:1001F000D8A409EF01F04D3A4C380F0B4D264C387E
:10020000F00B4C6E4B380F0B4C264B38F00B4B6EF3
:100210005984D8904DBECEEF00F04B364C364D365B
:10022000592A4DBECEEF00F04B364C364D36592A8A
:100230004DBECEEF00F04B364C364D36592ACEEF40
:1002400000F04CC04DF04BC04CF04B6A000E59967C
:1002500059884D644EEF01F0F00E4D14D8A439EFDB
:1002600001F04D3A4C380F0B4D264C38F00B4C6ECC
:100270005984D8904DBECEEF00F04C364D36592AF9
:100280004DBECEEF00F04C364D36592A4DBECEEF66
:1002900000F04C364D36592ACEEF00F04CC04DF0F0
:1002A0004C6A000E59864D6481EF01F0F00E4D143A
:1002B000D8A45DEF01F04D3A5984D8904DBECEEFF1
:1002C00000F04D36592A4DBECEEF00F04D36592A7A
:1002D0004DBECEEF00F04D36592ACEEF00F0010EA4
:1002E000576E68EC00F085EF01F0020E576E76EC69
:1002F00000F085EF01F0040E576E7BEC00F085EF07
:1003000001F0080E576E88EC00F012000001586AE8
:10031000536A4B50D8B4000C4F18556E55BE581E3A
:10032000566A4FAE96EF01F04F1E4F2A4BA09BEF3F
:1003300001F04B1E4B2A4B504F10556E55BEC2EF6D
:1003400001F04F50535E4B364B3453364F505326CB
:100350004B36060E576E4B3453364F504BB0535EF0
:100360004BA053264B36572EABEF01F04BA0532634
:1003700056B0D4EF01F058AE000C4B1E4B2A531E62
:10038000532A000C4FAED0EF01F04BBECDEF01F081
:100390004B50536E4B6ABBEF01F04B6A4B2A000C7B
:1003A0004B1E562AA1EF01F0532A4F50535CD8A49C
:1003B000BBEF01F0536A4B2A4BAEBBEF01F0FF0CD1
:1003C00012000001536A546A000E52624E6467EFD5
:1003D00002F04D505118556E52504E267E0ED8A048
:1003E000F8EF01F04E5ED8B06CEF02F0FCEF01F0D8
:1003F0004E5ED8A071EF02F04D8E518E4DC059F077
:100400004CC056F04BC058F04B504F02F4CF57F051
:100410004C505002F4CF4BF0F3CF53F04F02F35057
:100420005726F4505322000E4B2258505002F350DE
:100430005726F4505322000E4B224D504F02F350DA
:100440005326F4504B224D5050024C6A000E4C2261
:10045000F3504B26F4504C2258505102F35053267F
:10046000F4504B224D6A000E4C224D225650510240
:10047000F3504B26F4504C22000E4D22595051029D
:10048000F3504C26F4504D224DBE4FEF02F0533640
:100490004B364C364D364E06D8B471EF02F062EF53
:1004A00002F0D880800E53644B30000E4B224C2259
:1004B0004D22D8A062EF02F04D324C324B324E4A00
:1004C0006CEF02F055AE4D9E000E74EF02F0010E7F
:1004D00088EC00F074EF02F0020E7BEC00F074EF99
:1004E00002F0040E68EC00F012000001536B080EDD
:1004F000576E4B3453364F50535ED8B082EF02F0F4
:100500005326D8904B36572E79EF02F01200000197
:100510004C34533654364F50535E5050D8A0503C54
:10052000545E4B364C360F0E576E4C3453365436A1
:100530004F504BA0A3EF02F0535E5050D8A0503C58
:10054000545EA8EF02F053265050D8B0503C5426C9
:100550004B364C36572E95EF02F04BB0B6EF02F00B
:100560004F5053265050D8B0503C54260000120033
:100570000001566A5686FF0E12000001568056AEE4
:10058000CAEF02F04D6A55AEFF0E4D6E4C6E4B6ECB
:1005900055364D32FF0E120000014D505118596E64
:1005A000536A546A566A4E505264C0EF03F0515079
:1005B000556E518E4D8E4E50566E52504E6E000EF0
:1005C000566410EF03F05650525ED8B4B1EF03F00A
:1005D000070E52647FEF03F0525E4BC053F04CC0E5
:1005E0004BF04DC04CF04D6A524EB1EF03F05264E7
:1005F00054EF03F0525E4BC053F04CC04BF04C6ACA
:10060000524EB1EF03F0526432EF03F0525E4BC032
:1006100053F04B6A524EB1EF03F0526419EF03F0FE
:1006200055C04DF050C04CF04FC04BF0536ADDEF59
:1006300004F0030E526424EF03F0525E53380F0BA4
:10064000536E524EB1EF03F0D8905332524EB1EF89
:1006500003F0D8905332524EB1EF03F0D89053329A
:10066000B1EF03F0030E526443EF03F0525E5338D0
:100670000F0B536E4B38F00B53264B380F0B4B6E52
:10068000524EB1EF03F0D8904B325332524EB1EF8D
:1006900003F0D8904B325332524EB1EF03F0D89062
:1006A0004B325332B1EF03F0030E52646BEF03F0A1
:1006B000525E53380F0B536E4B38F00B53264B38AA
:1006C0000F0B4B6E4C38F00B4B264C380F0B4C6E0F
:1006D000524EB1EF03F0D8904C324B325332524E5F
:1006E000B1EF03F0D8904C324B325332524EB1EF4F
:1006F00003F0D8904C324B325332B1EF03F0030E7B
:1007000052649CEF03F0525E53380F0B536E4B381C
:10071000F00B53264B380F0B4B6E4C38F00B4B261F
:100720004C380F0B4C6E4D38F00B4C264D380F0BE0
:100730004D6E524EB1EF03F0D8904D324C324B32E9
:100740005332524EB1EF03F0D8904D324C324B320F
:100750005332524EB1EF03F0D8904D324C324B32FF
:100760005332546A000E59AEA5EF04F0531E4B1ECF
:100770004C1E4D1E532A4B224C224D22A5EF04F055
:100780005250D8A4C6EF03F0DDEF04F0546A4DC018
:1007900055F04D8E518E52504E5C526ED8B498EF3B
:1007A00004F0070E526466EF04F0525E4F50546E30
:1007B00050504F6E5150506E516A524E98EF04F0A7
:1007C000070E52643BEF04F0525E4F50546E50508F
:1007D0004F6E506A524E98EF04F0070E526419EFB4
:1007E00004F0525E4F50546E4F6A524E98EF04F030
:1007F000070E526400EF04F055C04DF0DDEF04F039
:10080000030E52640BEF04F0525E54380F0B546E1B
:10081000524E98EF04F0D8905432524E98EF04F0B4
:10082000D8905432524E98EF04F0D890543298EF4A
:1008300004F0030E52642AEF04F0525E54380F0B9A
:10084000546E4F38F00B54264F380F0B4F6E524EEC
:1008500098EF04F0D8904F325432524E98EF04F093
:10086000D8904F325432524E98EF04F0D8904F3215
:10087000543298EF04F0030E526452EF04F0525ECB
:1008800054380F0B546E4F38F00B54264F380F0B63
:100890004F6E5038F00B4F2650380F0B506E524EA3
:1008A00098EF04F0D89050324F325432524E98EFB5
:1008B00004F0D89050324F325432524E98EF04F038
:1008C000D89050324F32543298EF04F0030E5264F5
:1008D00083EF04F0525E54380F0B546E4F38F00B18
:1008E00054264F380F0B4F6E5038F00B4F265038B0
:1008F0000F0B506E5138F00B502651380F0B516EC4
:10090000524E98EF04F0D890513250324F32543258
:10091000524E98EF04F0D890513250324F32543248
:10092000524E98EF04F0D890513250324F32543238
:10093000536A000E59AEA5EF04F0541E4F1E501E10
:10094000511E542A4F2250225122545053264F50A8
:100950004B2250504C2251504D2259BEBCEF04F056
:10096000D8A0CBEF04F04D324C324B3253324E3ED6
:10097000CBEF04F0D7EF04F0D8B0D1EF04F0000EC5
:10098000531E4B1E4C1E4D1E532A4B224C224D22F1
:10099000557ED1EF04F0010E576E90EC00F0DFEFC2
:1009A00004F0020E576E90EC00F0DFEF04F0040E3E
:1009B000576E7BEC00F0DFEF04F0000E576E120074
:1009C00000001200080E566EFF0E556E562E01D016
:1009D00003D0552EFED7FAD71E0E556E552EFED7D4
:1009E0001200100E556E552EFED7000012000101A8
:1009F0005651390807E3300E565D04E3010E4B6E85
:100A000003EF05F04B6A1200800E010156194B6E80
:100A1000800E000A4B5CD8B075D1565100084F6E5D
:100A20004FC056F1800E4F184B6E800E6E0A4B5C15
:100A3000D8A0C0D0640E4F6E56C14BF086EC01F0CA
:100A4000120E4B26000E4BBEFF0E4C6E000E4C22BB
:100A5000020E4F6E000E4CBEFF0E4D6E4E6E4F508E
:100A600007E04B364B904C364D364E36FF0FF8D7DD
:100A7000280E4B264B0E4C22000E4D224BC0F6FF8B
:100A80004CC0F7FF4DC0F8FF0900F5CF57F1090042
:100A9000F5CF58F10900F5CF59F10900F5CF5AF11A
:100AA000640E4F6E56C14BF086EC01F053C04BF014
:100AB0000A0E4F6E86EC01F0090E4B26000E4BBE5F
:100AC000FF0E4C6E000E4C22020E4F6E000E4CBEFE
:100AD000FF0E4D6E4E6E4F5007E04B364B904C362E
:100AE0004D364E36FF0FF8D7280E4B264B0E4C22B4
:100AF000000E4D224BC0F6FF4CC0F7FF4DC0F8FF73
:100B00000900F5CF4BF00900F5CF4CF00900F5CF07
:100B10004DF00900F5CF4EF057C14FF058C150F0DD
:100B200059C151F05AC152F0E1EC01F04BC057F1FC
:100B30004CC058F14DC059F14EC05AF10A0E4F6EDB
:100B400056C14BF086EC01F053C04BF0020E4F6ED5
:100B5000000E4BBEFF0E4C6E4D6E4E6E4F5007E0BA
:100B60004B364B904C364D364E36FF0FF8D7280E8D
:100B70004B264B0E4C22000E4D224BC0F6FF4CC0B4
:100B8000F7FF4DC0F8FF0900F5CF4BF00900F5CF96
:100B90004CF00900F5CF4DF00900F5CF4EF057C1EC
:100BA0004FF058C150F059C151F05AC152F0E1EC28
:100BB00001F01200800E0A0A4B6E800E01015619D8
:100BC0004B5C72E20A0E4F6E56C14BF086EC01F0A0
:100BD000090E4B26000E4BBEFF0E4C6E000E4C2233
:100BE000020E4F6E000E4CBEFF0E4D6E4E6E4F50FD
:100BF00007E04B364B904C364D364E36FF0FF8D74C
:100C0000280E4B264B0E4C22000E4D224BC0F6FFF9
:100C10004CC0F7FF4DC0F8FF0900F5CF57F10900B0
:100C2000F5CF58F10900F5CF59F10900F5CF5AF188
:100C30000A0E4F6E56C14BF086EC01F053C04BF0DC
:100C4000020E4F6E000E4BBEFF0E4C6E4D6E4E6E82
:100C50004F5007E04B364B904C364D364E36FF0F1B
:100C6000F8D7280E4B264B0E4C22000E4D224BC0BF
:100C7000F6FF4CC0F7FF4DC0F8FF0900F5CF4BF071
:100C80000900F5CF4CF00900F5CF4DF00900F5CF84
:100C90004EF057C14FF058C150F059C151F05AC1F0
:100CA00052F0E1EC01F012000001020E4F6E56C14D
:100CB0004BF0000E010156BFFF0E4C6E4D6E4E6E96
:100CC0004F5007E04B364B904C364D364E36FF0FAB
:100CD000F8D7280E4B264B0E4C22000E4D224BC04F
:100CE000F6FF4CC0F7FF4DC0F8FF0900F5CF4BF001
:100CF0000900F5CF4CF00900F5CF4DF00900F5CF14
:100D00004EF01200800E010156194B6E800E6E0AD5
:100D10004B5CD8A0C0D0640E4F6E56C14BF086EC31
:100D200001F0120E4B26000E4BBEFF0E4C6E000E55
:100D30004C22020E4F6E000E4CBEFF0E4D6E4E6EDC
:100D40004F5007E04B364B904C364D364E36FF0F2A
:100D5000F8D75C0E4B264B0E4C22000E4D224BC09A
:100D6000F6FF4CC0F7FF4DC0F8FF0900F5CF57F173
:100D70000900F5CF58F10900F5CF59F10900F5CF79
:100D80005AF1640E4F6E56C14BF086EC01F053C021
:100D90004BF00A0E4F6E86EC01F0090E4B26000E4A
:100DA0004BBEFF0E4C6E000E4C22020E4F6E000E1C
:100DB0004CBEFF0E4D6E4E6E4F5007E04B364B90C3
:100DC0004C364D364E36FF0FF8D75C0E4B264B0E89
:100DD0004C22000E4D224BC0F6FF4CC0F7FF4DC019
:100DE000F8FF0900F5CF4BF00900F5CF4CF00900F2
:100DF000F5CF4DF00900F5CF4EF057C14FF058C177
:100E000050F059C151F05AC152F0E1EC01F04BC021
:100E100057F14CC058F14DC059F14EC05AF10A0E6D
:100E20004F6E56C14BF086EC01F053C04BF0020EF2
:100E30004F6E000E4BBEFF0E4C6E4D6E4E6E4F5001
:100E400007E04B364B904C364D364E36FF0FF8D7F9
:100E50005C0E4B264B0E4C22000E4D224BC0F6FF73
:100E60004CC0F7FF4DC0F8FF0900F5CF4BF009006B
:100E7000F5CF4CF00900F5CF4DF00900F5CF4EF05D
:100E800057C14FF058C150F059C151F05AC152F0FA
:100E9000E1EC01F01200800E0A0A4B6E800E010197
:100EA00056194B5C72E20A0E4F6E56C14BF086EC3F
:100EB00001F0090E4B26000E4BBEFF0E4C6E000ECD
:100EC0004C22020E4F6E000E4CBEFF0E4D6E4E6E4B
:100ED0004F5007E04B364B904C364D364E36FF0F99
:100EE000F8D75C0E4B264B0E4C22000E4D224BC009
:100EF000F6FF4CC0F7FF4DC0F8FF0900F5CF57F1E2
:100F00000900F5CF58F10900F5CF59F10900F5CFE7
:100F10005AF10A0E4F6E56C14BF086EC01F053C0E9
:100F20004BF0020E4F6E000E4BBEFF0E4C6E4D6E20
:100F30004E6E4F5007E04B364B904C364D364E368A
:100F4000FF0FF8D75C0E4B264B0E4C22000E4D22A5
:100F50004BC0F6FF4CC0F7FF4DC0F8FF0900F5CFBE
:100F60004BF00900F5CF4CF00900F5CF4DF009002A
:100F7000F5CF4EF057C14FF058C150F059C151F064
:100F80005AC152F0E1EC01F012000001020E4F6E66
:100F900056C14BF0000E010156BFFF0E4C6E4D6E58
:100FA0004E6E4F5007E04B364B904C364D364E361A
:100FB000FF0FF8D75C0E4B264B0E4C22000E4D2235
:100FC0004BC0F6FF4CC0F7FF4DC0F8FF0900F5CF4E
:100FD0004BF00900F5CF4CF00900F5CF4DF00900BA
:100FE000F5CF4EF012006E0E0101565DD8A0CAD0AA
:100FF000640E4F6E56C14BF075EC02F0120E4B268C
:101000004C6A000E4C22020E4F6E000E4CBEFF0EBC
:101010004D6E4E6E4F5007E04B364B904C364D3672
:101020004E36FF0FF8D7280E4B264B0E4C22000EE3
:101030004D224BC0F6FF4CC0F7FF4DC0F8FF090032
:10104000F5CF4BF00900F5CF4CF00900F5CF4DF08E
:101050000900F5CF4EF0000E4F6E000E506E000EE0
:10106000516E7E0E526EE1EC01F04BC057F14CC058
:1010700058F14DC059F14EC05AF1640E4F6E56C131
:101080004BF075EC02F053C04BF00A0E4F6E75EC4E
:1010900002F0090E4B264C6A000E4C22020E4F6ED7
:1010A000000E4CBEFF0E4D6E4E6E4F5007E04B369D
:1010B0004B904C364D364E36FF0FF8D7280E4B2648
:1010C0004B0E4C22000E4D224BC0F6FF4CC0F7FFDA
:1010D0004DC0F8FF0900F5CF4BF00900F5CF4CF0FB
:1010E0000900F5CF4DF00900F5CF4EF057C14FF094
:1010F00058C150F059C151F05AC152F0E1EC01F021
:101100004BC057F14CC058F14DC059F14EC05AF187
:101110000A0E4F6E56C14BF075EC02F053C04BF007
:10112000020E4F6E000E4C6E4D6E4E6E4F5007E02D
:101130004B364B904C364D364E36FF0FF8D7280EB7
:101140004B264B0E4C22000E4D224BC0F6FF4CC0DE
:10115000F7FF4DC0F8FF0900F5CF4BF00900F5CFC0
:101160004CF00900F5CF4DF00900F5CF4EF057C116
:101170004FF058C150F059C151F05AC152F0E1EC52
:1011800001F01200010156510A08D8B07FD00A0EB2
:101190004F6E56C14BF075EC02F0090E4B264C6AAF
:1011A000000E4C22020E4F6E000E4CBEFF0E4D6E16
:1011B0004E6E4F5007E04B364B904C364D364E3608
:1011C000FF0FF8D7280E4B264B0E4C22000E4D2257
:1011D0004BC0F6FF4CC0F7FF4DC0F8FF0900F5CF3C
:1011E0004BF00900F5CF4CF00900F5CF4DF00900A8
:1011F000F5CF4EF0000E4F6E000E506E000E516E89
:101200007E0E526EE1EC01F04BC057F14CC058F12C
:101210004DC059F14EC05AF10A0E4F6E56C14BF0F7
:1012200075EC02F053C04BF0020E4F6E000E4C6E88
:101230004D6E4E6E4F5007E04B364B904C364D3650
:101240004E36FF0FF8D7280E4B264B0E4C22000EC1
:101250004D224BC0F6FF4CC0F7FF4DC0F8FF090010
:10126000F5CF4BF00900F5CF4CF00900F5CF4DF06C
:101270000900F5CF4EF057C14FF058C150F059C199
:1012800051F05AC152F0E1EC01F012000001020EDF
:101290004F6E56C14BF0000E4C6E4D6E4E6E4F5061
:1012A00007E04B364B904C364D364E36FF0FF8D795
:1012B000280E4B264B0E4C22000E4D224BC0F6FF43
:1012C0004CC0F7FF4DC0F8FF0900F5CF4BF0090007
:1012D000F5CF4CF00900F5CF4DF00900F5CF4EF0F9
:1012E000000E4F6E000E506E000E516E7E0E526E4E
:1012F000E1EC01F0120000014B504F02F4CF54F02A
:10130000F3CF53F04C505002F4CF56F0F3CF55F0DA
:101310004B505002F3505426F4505522E86A56229E
:101320004C504F02F3505426F4505522E86A56228E
:1013300050AE9FEF09F04B50555C4C5056584CAE98
:10134000A6EF09F04F50555C5050565853C04BF023
:1013500054C04CF055C04DF056C04EF01200000184
:10136000556A4E50D8A455805250D8A45582555035
:10137000D8B413EF0AF0030AD8B4CCEF09F055B093
:10138000C7EF09F051AE11EF0AF00FEF0AF04DAEC2
:101390000FEF0AF011EF0AF04D50800B556E4D9E85
:1013A0005150800B519E5518D8B4DDEF09F05550BF
:1013B000D8B40FEF0AF011EF0AF052504E5CD8B4D7
:1013C000E7EF09F0D8A003EF0AF009EF0AF0515057
:1013D0004D5CD8B4F1EF09F0D8A003EF0AF009EFA3
:1013E0000AF050504C5CD8B4FBEF09F0D8A003EFE2
:1013F0000AF009EF0AF04F504B5CD8B413EF0AF033
:10140000D8B009EF0AF05552D8B411EF0AF00FEF37
:101410000AF05552D8B40FEF0AF011EF0AF0D88055
:101420001200D8901200D880D88412001200000157
:101430004E505218D8A42CEF0AF04D505118D8A491
:101440002CEF0AF04C505018D8A42CEF0AF04B5057
:101450004F18D8B4D8841200D8941200120000019A
:10146000586A546A536A4C504B10D8B4000C4C5014
:101470005018556E55BE581E566A50AE45EF0AF0CC
:101480004F1E501E4F2AD8B4502A4CAE4DEF0AF0D2
:101490004B1E4C1E4B2AD8B44C2A4C505010556E43
:1014A00055BE65EF0AF087EC02F056B07CEF0AF00B
:1014B00058AE000C4B1E4C1E4B2AD8B44C2A531E5F
:1014C000541E532AD8B4542A000C50AE77EF0AF0B9
:1014D0004CBE73EF0AF04C50546E4B50536E4C6A36
:1014E0004B6A58EF0AF04C6A4B6A4B2A000C4C1EB0
:1014F0004B1E562A53EF0AF0532AD8B4542A4F50A1
:10150000535CD8A458EF0AF05050545CD8A458EF5C
:101510000AF0546A536A4B2AD8B44C2A4CAE58EF9E
:101520000AF00000FF0C12000001536A546A525086
:10153000D8B42BEF0BF04E50D8B430EF0BF04D5029
:101540005118556E4D8E518E596A4DC053F04CC096
:1015500057F04BC058F04F50585E5050D8A0503CF8
:10156000575E5150D8A0513C535E536A576A586A2F
:10157000D8A0C2EF0AF0D8904D324C324B325332E1
:10158000010E596E52504E5ED8A0CFEF0AF07E0E7B
:1015900059244E26D8B035EF0BF0D5EF0AF07E0E69
:1015A00059244E26D8A03AEF0BF0180E566E583636
:1015B000573653364B364C364D3659364F504B5EB8
:1015C0005050D8A0503C4C5E5150D8A0513C4D5E7C
:1015D0005134591259A0F0EF0AF05880FBEF0AF08D
:1015E0004F504B265050D8B0503C4C265150D8B09C
:1015F00051284D265890562ED7EF0AF021EF0BF0C8
:10160000D8904B364C364D3659364F504B5E505075
:10161000D8A0503C4C5E5150D8A0513C4D5E513446
:101620005910010B5826D8B0572AD8B4532AD8A439
:1016300021EF0BF05332573258324E2AD8B435EFDF
:101640000BF055AE539E53504D6E57504C6E585044
:101650004B6E3DEF0BF0010EB8EC02F03DEF0BF0DE
:10166000020E88EC00F03DEF0BF0040E7BEC00F076
:101670003DEF0BF0080E68EC00F012000001566A16
:10168000576A556A536A4E50D8B4C7EF0BF04D8E67
:101690009E0E4E5E4EBE52EF0BF0D8B452EF0BF0E2
:1016A000B7EF0BF04E6C080E4E5CD8A084EF0BF039
:1016B0004E6E53364BC053F04CC04BF04DC04CF007
:1016C0004D6A080E4E5CD8A084EF0BF04E6E533678
:1016D0004BC053F04CC04BF04C6A080E4E5CD8A087
:1016E00084EF0BF04E6E53364BC053F04B6A080E2E
:1016F0004E5CD8A084EF0BF04E6E5336536A4E50BA
:10170000D8A4D89090EF0BF04E50D8B490EF0BF0D7
:10171000D8904D324C324B3253324E2E88EF0BF074
:1017200056BC53A0A1EF0BF0D8A0A1EF0BF0532AA9
:10173000D8B44B2AD8B44C2AD8B44D2A4DBECBEFDE
:101740000BF055AEC7EF0BF04D1E4C1E4B1E531E3B
:10175000532AD8B44B2AD8B44C2AD8B44D2AC7EF50
:101760000BF04D6A4C6A4B6A536AC7EF0BF0568018
:1017700056AED1EF0BF04D6A55AED1EF0BF04D6E7A
:101780004C6E4B6E536E55364D32D1EF0BF0000E52
:10179000576AD2EF0BF0010E576EBDEC02F0D2EF9C
:1017A0000BF0FF0E4D504E6E4C504D6E4B504C6E2C
:1017B00053504B6E120000014B50536E4C504B6E09
:1017C0004D504C6E4E504D6E4E6A566A576A9E0E84
:1017D0004E6E556A020E576E90EC00F0120000013A
:1017E000517ECCEC02F012000001566A556A546A30
:1017F000536A596A4E3453364F50535E5050D8A0F6
:10180000503C545E5150D8A0513C555E5250D8A027
:10181000523C565EE86AD8A0010E595E4E36070E5D
:10182000576E4E34533654365536563659364F5019
:101830004EA02EEF0CF0535E5050D8A0503C545E9A
:101840005150D8A0513C555E5250D8A0523C565EE3
:10185000E86AD8A0010E595E3FEF0CF053265050B5
:10186000D8B0503C54265150D8B0513C5526525017
:10187000D8B0523C5626E86AD8B0010E59264E36EA
:10188000572E11EF0CF04D3453365436553656362C
:1018900059364F504EA060EF0CF0535E5050D8A018
:1018A000503C545E5150D8A0513C555E5250D8A087
:1018B000523C565EE86AD8A0010E595E71EF0CF0FA
:1018C00053265050D8B0503C54265150D8B0513CBB
:1018D00055265250D8B0523C5626E86AD8B0010E70
:1018E00059264D36070E576E4D34533654365536FD
:1018F000563659364F504DA091EF0CF0535E505074
:10190000D8A0503C545E5150D8A0513C555E525026
:10191000D8A0523C565EE86AD8A0010E595EA2EFEC
:101920000CF053265050D8B0503C54265150D8B0EB
:10193000513C55265250D8B0523C5626E86AD8B091
:10194000010E59264D36572E74EF0CF04C34533699
:1019500054365536563659364F504DA0C3EF0CF01D
:10196000535E5050D8A0503C545E5150D8A0513CCA
:10197000555E5250D8A0523C565EE86AD8A0010E7F
:10198000595ED4EF0CF053265050D8B0503C54263A
:101990005150D8B0513C55265250D8B0523C5626E2
:1019A000E86AD8B0010E59264C36070E576E4C34F3
:1019B000533654365536563659364F504CA0F4EF00
:1019C0000CF0535E5050D8A0503C545E5150D8A0FB
:1019D000513C555E5250D8A0523C565EE86AD8A0A1
:1019E000010E595E05EF0DF053265050D8B0503C13
:1019F00054265150D8B0513C55265250D8B0523C84
:101A00005626E86AD8B0010E59264C36572ED7EF25
:101A10000CF04B34533654365536563659364F50F3
:101A20004CA026EF0DF0535E5050D8A0503C545EB1
:101A30005150D8A0513C555E5250D8A0523C565EF1
:101A4000E86AD8A0010E595E37EF0DF053265050CA
:101A5000D8B0503C54265150D8B0513C5526525025
:101A6000D8B0523C5626E86AD8B0010E59264B36FB
:101A7000070E576E4B345336543655365636593654
:101A80004F504BA057EF0DF0535E5050D8A0503C34
:101A9000545E5150D8A0513C555E5250D8A0523C93
:101AA000565EE86AD8A0010E595E68EF0DF0532625
:101AB0005050D8B0503C54265150D8B0513C5526C7
:101AC0005250D8B0523C5626E86AD8B0010E59267A
:101AD0004B36572E3AEF0DF04BB07DEF0DF04F50D7
:101AE00053265050D8B0503C54265150D8B0513C99
:101AF00055265250D8B0523C562612000001566A64
:101B0000576A536A4E50D8B403EF0EF04DC055F0EB
:101B10004D8E9E0E4E5E4EAEF3EF0DF04E6C080EE7
:101B20004E5CD8A0C0EF0DF04E6E53364BC053F054
:101B30004CC04BF04DC04CF04D6A080E4E5CD8A026
:101B4000C0EF0DF04E6E53364BC053F04CC04BF00F
:101B50004C6A080E4E5CD8A0C0EF0DF04E6E5336A6
:101B60004BC053F04B6A080E4E5CD8A0C0EF0DF08E
:101B70004E6E5336536A4E50D8A4D890CCEF0DF029
:101B80004E50D8B4CCEF0DF0D8904D324C324B3291
:101B900053324E2EC4EF0DF056BC53A0DDEF0DF0C6
:101BA000D8A0DDEF0DF0532AD8B44B2AD8B44C2A74
:101BB000D8B44D2A4DBE07EF0EF055AE03EF0EF030
:101BC0004D1E4C1E4B1E531E532AD8B44B2AD8B45C
:101BD0004C2AD8B44D2A03EF0EF04D6A4C6A4B6A7A
:101BE000536A03EF0EF0568056AE0EEF0EF04D6ABC
:101BF00055AE0EEF0EF04D6E4C6E4B6E536E55366D
:101C00004D320EEF0EF0576A000E0FEF0EF0010E80
:101C1000576E000EBDEC02F00FEF0EF0FF0E4D50B0
:101C20004E6E4C504D6E4B504C6E53504B6E1200DE
:101C300009500A1000E009C0E9FF0AC0EAFF0101EB
:101C4000565300E0EF96EF9EEF9CEF9AEF98EF94DB
:101C500056BFEF8E56BDEF8C56BBEF8A56B9EF8854
:101C60000B50010A03E1EF9437EF0EF0EF84EF869B
:101C7000E0EC04F00101565300E0EF96EF9EEF9C7C
:101C8000EF9AEF98EF9456B7EF8E56B5EF8C56B3A8
:101C9000EF8A56B1EF880B50010A03E1EF9452EF3F
:101CA0000EF0EF84EF86E0EC04F0EF960B50010AA3
:101CB00003E1E2EC04F002D0F1EC04F01200280E93
:101CC0000101346F6E0E356F750E366F6C0E376F07
:101CD0006C0E386F290E396F3A6B426B436B406B59
:101CE000416B2FC14BF030C14CF031C14DF0010EB2
:101CF00001012F27000E302331234BC0F6FF4CC0CB
:101D0000F7FF4DC0F8FF0900F5CF4BF04BC03DF198
:101D10004B52D8B495EF1FF03D51250A0BE02DC171
:101D2000E1FF2EC1E2FF3DC1E6FF2D4B2E2B424BC2
:101D3000432BD7D701013E6B3F6B406B416B28D0E3
:101D400001014087010E2F27000E302331235ED082
:101D500001014081010E2F27000E3023312356D080
:101D600001014083010E2F27000E302331234ED076
:101D700001014187010E2F27000E3023312346D069
:101D800001014085010E2F27000E302331233ED064
:101D90002FC1F6FF30C1F7FF31C1F8FF0900F5CFC1
:101DA0004EF101014E512D0ACBE02FC1F6FF30C19B
:101DB000F7FF31C1F8FF0900F5CF4EF14E51200A6F
:101DC000C7E02FC1F6FF30C1F7FF31C1F8FF0900AE
:101DD000F5CF4EF14E512B0AC3E02FC1F6FF30C1B3
:101DE000F7FF31C1F8FF0900F5CF4EF14E51230A3C
:101DF000BFE02FC1F6FF30C1F7FF31C1F8FF090086
:101E0000F5CF4EF14E51300ABBE001D098D7010119
:101E100040B34091010140B740952FC1F6FF30C15A
:101E2000F7FF31C1F8FF0900F5CF4BF0000E4C6E03
:101E30004BC056F1F7EC04F04B5238E001013E6B19
:101E40003F6B3EC14BF03FC14CF00A0E4F6E000E8F
:101E5000506E7BEC09F02FC1F6FF30C1F7FF31C1A6
:101E6000F8FF0900F5CF4EF101014E514B243E6FB2
:101E7000000E4C203F6F300E3E5F000E3F5B010EA8
:101E80002F27000E302331232FC1F6FF30C1F7FF7B
:101E900031C1F8FF0900F5CF4BF0000E4C6E4BC07E
:101EA00056F1F7EC04F04B52CCE136D02FC1F6FFDF
:101EB00030C1F7FF31C1F8FF0900F5CF4EF1010144
:101EC0004E512A0A29E132C1E9FF33C1EAFFEECFC0
:101ED0004BF0EECF4CF04BC0E9FF4CC0EAFFEECF29
:101EE0003EF1EECF3FF132C1E9FF33C1EAFFEECF61
:101EF0004BF0EECF4CF0020E4B26000E4C2232C1BE
:101F0000E1FF33C1E2FF4BC0E6FF4CC0E6FF010E2C
:101F10002F27000E302331232FC1F6FF30C1F7FFEA
:101F200031C1F8FF0900F5CF4EF101014E512E0AE3
:101F300075E1010E2F27000E302331232FC1F6FF4C
:101F400030C1F7FF31C1F8FF0900F5CF4EF14E5116
:101F50002A0A2AE132C1E9FF33C1EAFFEECF4BF092
:101F6000EECF4CF04BC0E9FF4CC0EAFFEECF3BF1A7
:101F7000EECF3CF132C1E9FF33C1EAFFEECF4BF0C7
:101F8000EECF4CF0020E4B26000E4C2232C1E1FF88
:101F900033C1E2FF4BC0E6FF4CC0E6FF010E2F2726
:101FA000000E3023312338D001013B6B3C6B2FC135
:101FB000F6FF30C1F7FF31C1F8FF0900F5CF4BF054
:101FC000000E4C6E4BC056F1F7EC04F04B5224E07F
:101FD0003BC14BF03CC14CF00A0E4F6E000E506EF0
:101FE0007BEC09F02FC1F6FF30C1F7FF31C1F8FFDC
:101FF0000900F5CF4EF101014E514B243B6F000E0D
:102000004C203C6F300E3B5F000E3C5B010E2F27D7
:10201000000E30233123CBD7010104D001013B6BEB
:102020003C6B41892FC14BF030C14CF031C14DF0B8
:10203000010E01012F27000E302331234BC0F6FF84
:102040004CC0F7FF4DC0F8FF0900F5CF3DF101D1BD
:1020500042C14BF043C14CF0120001014089E2D76C
:102060000101418532D10101408B010141812DD116
:10207000010141832AD10101408D27D126D10101DF
:10208000408B0101408F21D132C1E9FF33C1EAFF0A
:10209000EECF4BF0EECF4CF04BC0E9FF4CC0EAFF67
:1020A000EECF4AF1EECF4BF132C1E9FF33C1EAFF87
:1020B000EECF4BF0EECF4CF0020E4B26000E4C2232
:1020C00032C1E1FF33C1E2FF4BC0E6FF4CC0E6FF87
:1020D000000E01014B1902E1000E4A1905E1340E10
:1020E00001014A6F010E4B6F01014C6B4D6B0101F9
:1020F0004C514A25E96E4D514B21EA6EEECF4BF023
:102100004B5203E04C4B4D2BF2D701013B513C119C
:102110000AE04D513C5D02E14C513B5D04E23BC1A4
:102120004CF13CC14DF101013F514D5D02E13E5189
:102130004C5D06E201014C513E5F4D513F5B03D0C7
:1021400001013E6B3F6B010140B717D03EC14BF020
:102150003FC14CF0010E01013E5F000E3F5B4B5052
:102160004C100BE02DC1E1FF2EC1E2FF200EE66E08
:102170002D4B2E2B424B432BE9D74CC14BF04DC17D
:102180004CF0010E01014C5F000E4D5B4B504C10AA
:1021900013E04AC1E9FF4BC1EAFFEECF4BF02DC17E
:1021A000E1FF2EC1E2FF4BC0E6FF2D4B2E2B4A4B29
:1021B0004B2B424B432BE1D7010140A717D03EC127
:1021C0004BF03FC14CF0010E01013E5F000E3F5B42
:1021D0004B504C100BE02DC1E1FF2EC1E2FF200E51
:1021E000E66E2D4B2E2B424B432BE9D77AD532C1CD
:1021F000E9FF33C1EAFFEECF4BF0EECF4CF04BC01E
:10220000E9FF4CC0EAFFEECF3DF132C1E9FF33C137
:10221000EAFFEECF4BF0EECF4CF0020E4B26000E55
:102220004C2232C1E1FF33C1E2FF4BC0E6FF4CC09C
:10223000E6FF3D0E01014A6F010E4B6F010E4C6F20
:10224000000E4D6F62D7C00E01014013000E411306
:102250003CD001013D51000AD8B4FAD63D516C0A78
:10226000D8B4FBD63D51660AD8B4FAD63D51450ADA
:10227000D8B4F9D63D51650AD8B4F7D63D51670AAE
:10228000D8B4F6D63D516F0AD8B4F5D63D51640A9C
:10229000D8B4F4D63D51690AD8B4F0D63D51700A8D
:1022A000D8B4EDD63D51580AD8B4E9D63D51780A94
:1022B000D8B4E7D63D51730AD8B4E6D63D51630A87
:1022C00096E03D51750ABFE0B4D7000E01014015FC
:1022D0004B6E4151070B4C6E4B504C10D8B4ECEF89
:1022E0001AF041A904D0060E3B6F000E3C6F32C1BC
:1022F000E9FF33C1EAFFEECF4BF0EECF4CF04BC01D
:10230000E9FF4CC0EAFFEECF44F1EECF45F1EECF4E
:1023100046F1EECF47F132C1E9FF33C1EAFFEECF1C
:102320004BF0EECF4CF0040E4B26000E4C2232C187
:10233000E1FF33C1E2FF4BC0E6FF4CC0E6FF4F6A4E
:10234000506A516A526A44C14BF045C14CF046C1D3
:102350004DF047C14EF0AFEC09F0010ED8B0000EC1
:102360004B6E4B5206E00101467F030E4013000EF8
:1023700041130101486B496B44C14BF045C14CF01E
:1023800046C14DF047C14EF04F6A506A516A526AD9
:1023900017EC0AF0000ED8A4010E4B6E4B52D8B4C5
:1023A00099D047C14BF04C6A4D6A4E6AFF0E4B14F0
:1023B0000101526F000E536F000E53177E0E4E6FC9
:1023C000000E4F6F506F516F4E51525D4B6E4F511B
:1023D00053594C6E4BC048F14CC049F1010E4B5C57
:1023E000486F000E4C58496F48C14BF049C14CF042
:1023F000030E4F6E000E506E7BEC09F04BC048F19F
:102400004CC049F10A0E4F6E000E506E2FEC0AF0D0
:102410004BC048F14CC049F1800E4C1801014E6F81
:10242000800E4E5D02E1000E4B5C04E2010E485F3F
:10243000000E495B48510008566F04EC05F044C19A
:102440004FF045C150F046C151F047C152F0E1ECA8
:1024500001F04BC04AF14CC04BF14DC04CF14EC0A5
:102460004DF1000E4F6E000E506E000E516E7F0E3D
:10247000526E4AC14BF04BC14CF04CC14DF04DC1B6
:102480004EF0AFEC09F0010ED8B0000E4B6E4B527F
:1024900006E0010E0101485F000E495B1BD0000EF3
:1024A0004F6E000E506E200E516E820E526E4AC15B
:1024B0004BF04BC14CF04CC14DF04DC14EF0AFEC68
:1024C00009F0000ED8B0010E4B6E4B5203E0010133
:1024D000484B492B0101800E4B6E800E01014919BA
:1024E0004B5C02E14851000804E3010E01013D6F1D
:1024F00002D048C13DF1010141B119D041A315D02D
:10250000800E49194B6E7F0E4B5C02E1FC0E485D5C
:102510000BE3800E010149194B6E800E3C194B5C98
:1025200002E13B51485D01E302D0E2EF16F0010108
:102530003B513C1107E041A305D0010E01013B5F77
:10254000000E3C5B000E4B6E01013C514B5C02E106
:102550003B51080804E2080E01013D6F02D03BC167
:102560003DF144C14BF045C14CF046C14DF047C16F
:102570004EF04F6A506A516A526A17EC0AF0000E28
:10258000D8A4010E4B6E4B52D8B460D148C156F15D
:1025900004EC05F04BC04FF04CC050F04DC051F072
:1025A0004EC052F044C14BF045C14CF046C14DF015
:1025B00047C14EF094EC0AF04BC044F14CC045F1D9
:1025C0004DC046F14EC047F101013D510008566F24
:1025D00004EC05F04BC04FF04CC050F04DC051F032
:1025E0004EC052F044C14BF045C14CF046C14DF0D5
:1025F00047C14EF094EC0AF04BC04EF14CC04FF185
:102600004DC050F14EC051F14EC144F14FC145F1A2
:1026100050C146F151C147F14EC14BF04FC14CF092
:1026200050C14DF051C14EF03EEC0BF0DBEC0BF025
:102630004BC04FF04CC050F04DC051F04EC052F066
:102640004EC14BF04FC14CF050C14DF051C14EF056
:10265000EFEC0BF0000E4F6E000E506E000E516E40
:102660007E0E526EAFEC09F0000ED8B0010E4B6E2C
:102670004B521AE044C14BF045C14CF046C14DF0FD
:1026800047C14EF0000E4F6E000E506E000E516EA0
:102690007E0E526ECCEC02F04BC044F14CC045F1C2
:1026A0004DC046F14EC047F144C14BF045C14CF01E
:1026B00046C14DF047C14EF03EEC0BF04BC052F11D
:1026C0004CC053F14DC054F14EC055F101013D5184
:1026D000010F4B6E4C6A000E4C22020E4F6E000E24
:1026E0004CBEFF0E4D6E4E6E4F5007E04B364B907A
:1026F0004C364D364E36FF0FF8D7900E4B264B0E0C
:102700004C22000E4D224BC0F6FF4CC0F7FF4DC0CF
:10271000F8FF0900F5CF4EF10900F5CF4FF10900A0
:10272000F5CF50F10900F5CF51F15151555D08E158
:102730005051545D05E14F51535D02E14E51525DE0
:102740001EE344C14BF045C14CF046C14DF047C1BA
:102750004EF0CD0E4F6ECC0E506E4C0E516E7B0E69
:10276000526EE1EC01F04BC044F14CC045F14DC05C
:1027700046F14EC047F10101484B492B67D044C197
:102780004BF045C14CF046C14DF047C14EF03EEC18
:102790000BF04BC052F14CC053F14DC054F14EC040
:1027A00055F1020E4F6E3DC14BF0000E4C6E4D6E5A
:1027B0004E6E4F5007E04B364B904C364D364E36F2
:1027C000FF0FF8D7900E4B264B0E4C22000E4D22D9
:1027D0004BC0F6FF4CC0F7FF4DC0F8FF0900F5CF26
:1027E0004EF10900F5CF4FF10900F5CF50F1090086
:1027F000F5CF51F101015151555D08E15051545D42
:1028000005E14F51535D02E14E51525D1FE244C15B
:102810004BF045C14CF046C14DF047C14EF0000EA3
:102820004F6E000E506E200E516E820E526EE1EC15
:1028300001F04BC044F14CC045F14DC046F14EC0D3
:1028400047F1010E0101485F000E495B010141A300
:102850009AD041B798D0800E000A4B6E800E0101CD
:102860003C194B5C02E13B510A0805E20A0E0101EA
:102870003B6F000E3C6F44C14BF045C14CF046C16C
:102880004DF047C14EF03EEC0BF04BC04AF14CC04E
:102890004BF14DC04CF14EC04DF101014A514B116D
:1028A0004C114D1144E00A0E4F6E000E506E516EE9
:1028B000526E4AC14BF04BC14CF04CC14DF04DC172
:1028C0004EF0F4EC0BF053C04BF054C04CF055C03C
:1028D0004DF056C04EF0000E01014E6F4E1808E14B
:1028E0004E514D1805E14E514C1802E14B50000A73
:1028F0001EE1010E01013B5F000E3C5B0A0E4F6EB4
:10290000000E506E516E526E4AC14BF04BC14CF0EE
:102910004CC14DF04DC14EF0F4EC0BF04BC04AF100
:102920004CC04BF14DC04CF14EC04DF1B6D7800EAE
:1029300001013C194B6E800E4B5C02E13D513B5D49
:1029400022E201013B513D5D566F04EC05F04BC0A6
:102950004FF04CC050F04DC051F04EC052F044C149
:102960004BF045C14CF046C14DF047C14EF094ECE0
:102970000AF04BC044F14CC045F14DC046F14EC089
:1029800047F13BC13DF10001050E01013B254B6EB6
:10299000000E3C214C6E4B503E5F4C503F5B3B5118
:1029A0003C1102E141A705D0010E01013E5F000E7E
:1029B0003F5B030E010140154B6E41C14CF0000E10
:1029C0004C164B504C1004E0010E3E5F000E3F5B76
:1029D000010140A54DD040A31BD0010E40154B6E08
:1029E00041C14CF0000E4C164B504C1003E02D0E24
:1029F0004B6E02D02B0E4B6E2DC1E1FF2EC1E2FFBC
:102A00004BC0E6FF01012D4B2E2B424B432B15D023
:102A1000010E010140154B6E41C14CF0000E4C16E9
:102A20004B504C100AE02DC1E1FF2EC1E2FF200EF9
:102A3000E66E2D4B2E2B424B432B800E4B6E800EA1
:102A400001013F194B5C02E13E51000810E22DC12B
:102A5000E1FF2EC1E2FF300EE66E01012D4B2E2B61
:102A6000424B432B010E3E5F000E3F5BE6D750D03A
:102A7000010140B71AD0800E4B6E800E01013F1944
:102A80004B5C02E13E51000810E22DC1E1FF2EC176
:102A9000E2FF200EE66E01012D4B2E2B424B432B05
:102AA000010E3E5F000E3F5BE6D7010140A31BD045
:102AB000010E40154B6E41C14CF0000E4C164B50B0
:102AC0004C1003E02D0E4B6E02D02B0E4B6E2DC121
:102AD000E1FF2EC1E2FF4BC0E6FF01012D4B2E2B83
:102AE000424B432B15D0010E010140154B6E41C1E5
:102AF0004CF0000E4C164B504C100AE02DC1E1FF7B
:102B00002EC1E2FF200EE66E2D4B2E2B424B432BA7
:102B100044C14BF045C14CF046C14DF047C14EF0A9
:102B20003EEC0BF04BC04AF14CC04BF14DC04CF1A8
:102B30004EC04DF1020E4F6E3DC14BF0000E4C6E7B
:102B40004D6E4E6E4F5007E04B364B904C364D3627
:102B50004E36FF0FF8D7900E4B264B0E4C22000E30
:102B60004D224BC0F6FF4CC0F7FF4DC0F8FF0900E7
:102B7000F5CF4FF00900F5CF50F00900F5CF51F037
:102B80000900F5CF52F04AC14BF04BC14CF04CC19B
:102B90004DF04DC14EF0F4EC0BF0300E4B262DC134
:102BA000E1FF2EC1E2FF4BC0E6FF01012D4B2E2BB2
:102BB000424B432B3B513C1102E141A776D02DC142
:102BC000E1FF2EC1E2FF2E0EE66E01012D4B2E2BF2
:102BD000424B432B3D513B5F000E3C5B01013D539B
:102BE00052E03D07020E4F6E3DC14BF0000E4C6EA1
:102BF0004D6E4E6E4F5007E04B364B904C364D3677
:102C00004E36FF0FF8D7900E4B264B0E4C22000E7F
:102C10004D224BC0F6FF4CC0F7FF4DC0F8FF090036
:102C2000F5CF4FF00900F5CF50F00900F5CF51F086
:102C30000900F5CF52F04AC14BF04BC14CF04CC1EA
:102C40004DF04DC14EF0F4EC0BF00A0E4F6E000E3D
:102C5000506E516E526EF4EC0BF053C04BF054C0FA
:102C60004CF055C04DF056C04EF0300E4B262DC1E5
:102C7000E1FF2EC1E2FF4BC0E6FF01012D4B2E2BE1
:102C8000424B432BABD73B513C110FE02DC1E1FF31
:102C90002EC1E2FF300EE66E2D4B2E2B424B432B06
:102CA000010E3B5F000E3C5BEED740AB0BD02DC15D
:102CB000E1FF2EC1E2FF450EE66E2D4B2E2B424B5F
:102CC000432B0AD02DC1E1FF2EC1E2FF650EE66E57
:102CD0002D4B2E2B424B432B800E49194B6E800EF1
:102CE0004B5C02E1000E485D12E248510008486F5B
:102CF00049C149F1E86A49572DC1E1FF2EC1E2FF00
:102D00002D0EE66E2D4B2E2B424B432B0AD02DC1A0
:102D1000E1FF2EC1E2FF2B0EE66E2D4B2E2B424B18
:102D2000432B0A0E4F6E000E506E48C14BF049C146
:102D30004CF02FEC0AF0300E4B262DC1E1FF2EC1D6
:102D4000E2FF4BC0E6FF01012D4B2E2B424B432BE4
:102D50000A0E4F6E000E506E48C14BF049C14CF048
:102D60002FEC0AF053C04BF054C04CF0300E4B2601
:102D70002DC1E1FF2EC1E2FF4BC0E6FF01012D4B4B
:102D80002E2B424B432B40A71BD0800E4B6E800E48
:102D90003F194B5C02E13E51000812E22DC1E1FFF8
:102DA0002EC1E2FF200EE66E01012D4B2E2B424B71
:102DB000432B010E3E5F000E3F5B3E513F11EEE1A3
:102DC00071EF0EF0010141A3FFD0800E49194B6E47
:102DD000800E4B5C02E1000E485D0BE2010E01012A
:102DE000485D4B6E000E49594C6E4B503B5F4C504A
:102DF0003C5B44C14BF045C14CF046C14DF047C16E
:102E00004EF03EEC0BF04BC04AF14CC04BF14DC0C4
:102E10004CF14EC04DF1010E01013D6F01013D51DC
:102E20000A0A39E0020E4F6E3DC14BF0000E4C6EA7
:102E30004D6E4E6E4F5007E04B364B904C364D3634
:102E40004E36FF0FF8D7900E4B264B0E4C22000E3D
:102E50004D224BC0F6FF4CC0F7FF4DC0F8FF0900F4
:102E6000F5CF4EF10900F5CF4FF10900F5CF50F144
:102E70000900F5CF51F1010151514D5D08E150516B
:102E80004C5D05E14F514B5D02E14E514A5D03E35C
:102E900001013D2BC3D701013D513B5D526F000E37
:102EA0003C59536F52C13BF153C13CF14AC14BF005
:102EB0004BC14CF04CC14DF04DC14EF0DBEC0BF072
:102EC0004BC04FF04CC050F04DC051F04EC052F0CE
:102ED00044C14BF045C14CF046C14DF047C14EF0E6
:102EE000EFEC0BF04BC04EF14CC04FF14DC050F128
:102EF0004EC051F152C156F104EC05F04EC14FF0F5
:102F00004FC150F050C151F051C152F0E1EC01F00D
:102F1000000E4F6E000E506E000E516E7E0E526E01
:102F2000CCEC02F03EEC0BF04BC04AF14CC04BF144
:102F30004DC04CF14EC04DF101013B513C1144E0FC
:102F40000A0E4F6E000E506E516E526E4AC14BF01B
:102F50004BC14CF04CC14DF04DC14EF0F4EC0BF0B8
:102F600053C04BF054C04CF055C04DF056C04EF01D
:102F7000000E01014E6F4E1808E14E514D1805E14B
:102F80004E514C1802E14B50000A1EE10A0E4F6EE2
:102F9000000E506E516E526E4AC14BF04BC14CF058
:102FA0004CC14DF04DC14EF0F4EC0BF04BC04AF16A
:102FB0004CC04BF14DC04CF14EC04DF1010E010122
:102FC0003B5F000E3C5BB8D7800E4B6E800E01015C
:102FD0003C194B5C02E13B510C0816E33BC156F136
:102FE000F3EC07F044C14FF045C150F046C151F039
:102FF00047C152F0CCEC02F04BC044F14CC045F15B
:103000004DC046F14EC047F144C14BF045C14CF0B4
:1030100046C14DF047C14EF04F6A506A516A526A3C
:1030200017EC0AF0000ED8A4010E4B6E4B52D8B428
:1030300078D044C14BF045C14CF046C14DF047C17A
:103040004EF03EEC0BF0000E01014E6F4E1808E101
:103050004E514D1805E14E514C1802E14B50000AFB
:1030600060E1800E4B6E800E49194B5C02E14851C5
:10307000010857E248C156F104EC05F04BC04FF08F
:103080004CC050F04DC051F04EC052F044C14BF016
:1030900045C14CF046C14DF047C14EF094EC0AF0EA
:1030A0005F0E4F6E700E506E090E516E810E526E95
:1030B000AFEC09F0010ED8B0000E4B6E4B5206E09B
:1030C000090E0101485F000E495B05D0080E0101A1
:1030D000485F000E495B48C156F104EC05F04BC057
:1030E0004FF04CC050F04DC051F04EC052F044C1B2
:1030F0004BF045C14CF046C14DF047C14EF094EC49
:103100000AF03EEC0BF04BC04AF14CC04BF14DC005
:103110004CF14EC04DF10101446B456B466B476B62
:1031200039D044C14BF045C14CF046C14DF047C1C8
:103130004EF03EEC0BF04BC04AF14CC04BF14DC091
:103140004CF14EC04DF14AC14BF04BC14CF04CC15B
:103150004DF04DC14EF0DBEC0BF04BC04FF04CC0CE
:1031600050F04DC051F04EC052F044C14BF045C13B
:103170004CF046C14DF047C14EF0EFEC0BF04BC0A8
:1031800044F14CC045F14DC046F14EC047F101013C
:10319000486B496B010E3D6F3D510A0A37E0020E44
:1031A0004F6E3DC14BF0000E4C6E4D6E4E6E4F504B
:1031B00007E04B364B904C364D364E36FF0FF8D766
:1031C000900E4B264B0E4C22000E4D224BC0F6FFAC
:1031D0004CC0F7FF4DC0F8FF0900F5CF4EF10900D4
:1031E000F5CF4FF10900F5CF50F10900F5CF51F1BE
:1031F00051514D5D08E150514C5D05E14F514B5D22
:1032000002E14E514A5D02E33D2BC6D73D513B25BD
:103210004B6E000E3C214C6E48514B2649514C22BE
:103220004B503E5F4C503F5B41B703D03B513C118C
:1032300004E0010E3E5F000E3F5B030E40154B6E37
:1032400041C14CF0000E4C164B504C1004E0010EE6
:103250003E5F000E3F5B40A549D040A31AD0010E4F
:1032600040154B6E41C14CF0000E4C164B504C10AB
:1032700003E02D0E4B6E02D02B0E4B6E2DC1E1FFE5
:103280002EC1E2FF4BC0E6FF2D4B2E2B424B432BB2
:1032900014D0010E40154B6E41C14CF0000E4C167F
:1032A0004B504C100AE02DC1E1FF2EC1E2FF200E71
:1032B000E66E2D4B2E2B424B432B800E4B6E800E19
:1032C0003F194B5C02E13E5100080FE22DC1E1FFC6
:1032D0002EC1E2FF300EE66E2D4B2E2B424B432BC0
:1032E000010E3E5F000E3F5BE8D74AD040B718D0D2
:1032F000800E4B6E800E3F194B5C02E13E51000880
:103300000FE22DC1E1FF2EC1E2FF200EE66E2D4B34
:103310002E2B424B432B010E3E5F000E3F5BE8D746
:1033200040A31AD0010E40154B6E41C14CF0000E67
:103330004C164B504C1003E02D0E4B6E02D02B0E52
:103340004B6E2DC1E1FF2EC1E2FF4BC0E6FF2D4BBE
:103350002E2B424B432B14D0010E40154B6E41C116
:103360004CF0000E4C164B504C100AE02DC1E1FF02
:103370002EC1E2FF200EE66E2D4B2E2B424B432B2F
:103380003DC14BF03D074B5251E0020E4F6E3DC127
:103390004BF0000E4C6E4D6E4E6E4F5007E04B36AC
:1033A0004B904C364D364E36FF0FF8D7900E4B26CD
:1033B0004B0E4C22000E4D224BC0F6FF4CC0F7FFC7
:1033C0004DC0F8FF0900F5CF4FF00900F5CF50F0E0
:1033D0000900F5CF51F00900F5CF52F04AC14BF08A
:1033E0004BC14CF04CC14DF04DC14EF0F4EC0BF024
:1033F0000A0E4F6E000E506E516E526EF4EC0BF0D2
:1034000053C04BF054C04CF055C04DF056C04EF078
:10341000300E4B262DC1E1FF2EC1E2FF4BC0E6FF6F
:1034200001012D4B2E2B424B432BAAD7800E4B6E06
:10343000800E49194B5C02E1485100080FE22DC192
:10344000E1FF2EC1E2FF300EE66E2D4B2E2B424BDC
:10345000432B010E485F000E495BE8D7800E000A3F
:103460004B6E800E3C194B5C02E13B51080803E2B5
:10347000080E3D6F02D03BC13DF13D513B5F000E58
:103480003C5B3D5302E141A70AD02DC1E1FF2EC1B3
:10349000E2FF2E0EE66E2D4B2E2B424B432B3DC1F1
:1034A00056F104EC05F044C14FF045C150F046C15F
:1034B00051F047C152F0E1EC01F07EEC0DF04BC051
:1034C0004AF14CC04BF14DC04CF14EC04DF10101E1
:1034D0003D5352E03D07020E4F6E3DC14BF0000ED2
:1034E0004C6E4D6E4E6E4F5007E04B364B904C3647
:1034F0004D364E36FF0FF8D7900E4B264B0E4C2212
:10350000000E4D224BC0F6FF4CC0F7FF4DC0F8FF38
:103510000900F5CF4FF00900F5CF50F00900F5CFC5
:1035200051F00900F5CF52F04AC14BF04BC14CF0BD
:103530004CC14DF04DC14EF0F4EC0BF00A0E4F6E45
:10354000000E506E516E526EF4EC0BF053C04BF007
:1035500054C04CF055C04DF056C04EF0300E4B26C6
:103560002DC1E1FF2EC1E2FF4BC0E6FF01012D4B53
:103570002E2B424B432BABD73B513C110FE02DC1BF
:10358000E1FF2EC1E2FF300EE66E2D4B2E2B424B9B
:10359000432B010E3B5F000E3C5BEED740A71AD0D9
:1035A000800E4B6E800E3F194B5C02E13E510008CD
:1035B00011E22DC1E1FF2EC1E2FF200EE66E2D4B80
:1035C0002E2B424B432B010E3E5F000E3F5B3E51C4
:1035D0003F11EFE171EF0EF0C00E40154E6F41C18B
:1035E0004FF1000E4F17000E4F1902E1000E4E1959
:1035F000D8A481D040A929D032C1E9FF33C1EAFF64
:10360000EECF4BF0EECF4CF04BC0E9FF4CC0EAFFE1
:10361000EECF4AF1EECF4BF1EECF4CF1EECF4DF1C4
:1036200032C1E9FF33C1EAFFEECF4BF0EECF4CF0F1
:10363000040E4B26000E4C2232C1E1FF33C1E2FFE3
:103640004BC0E6FF4CC0E6FF2ED032C1E9FF33C1CC
:10365000EAFFEECF4BF0EECF4CF04BC0E9FF4CC091
:10366000EAFFEECF4AF1EECF4BF1000E4BBFFF0E5B
:103670004C6F4D6F000E4BBFFF0E4C6F4D6F32C144
:10368000E9FF33C1EAFFEECF4BF0EECF4CF0020E74
:103690004B26000E4C2232C1E1FF33C1E2FF4BC08A
:1036A000E6FF4CC0E6FF800E4D194B6E800E4B5C62
:1036B00008E1000E4C5D05E1000E4B5D02E1000EDD
:1036C0004A5D18E2030E4013000E41134B6A4C6A28
:1036D0004D6A4E6A4A514B5E4B514C5A4C514D5AB1
:1036E0004D514E5A4BC04AF14CC04BF14DC04CF1BC
:1036F0004EC04DF155D040A929D032C1E9FF33C1A8
:10370000EAFFEECF4BF0EECF4CF04BC0E9FF4CC0E0
:10371000EAFFEECF4AF1EECF4BF1EECF4CF1EECF18
:103720004DF132C1E9FF33C1EAFFEECF4BF0EECFEE
:103730004CF0040E4B26000E4C2232C1E1FF33C187
:10374000E2FF4BC0E6FF4CC0E6FF2AD032C1E9FFE2
:1037500033C1EAFFEECF4BF0EECF4CF04BC0E9FFA8
:103760004CC0EAFFEECF4AF1EECF4BF1000E4C6FAA
:103770004D6F000E4C6F4D6F32C1E9FF33C1EAFF50
:10378000EECF4BF0EECF4CF0020E4B26000E4C224B
:1037900032C1E1FF33C1E2FF4BC0E6FF4CC0E6FFA0
:1037A000000E3C1902E1000E3B190FE1000E4B6EBA
:1037B0004D1908E14B504C1905E14B504B1902E1F2
:1037C0004A51000A02E13B4B3C2BC00E40154B6EA8
:1037D0004BC052F1B7D0010E3D6F3D510A0A37E0A0
:1037E000020E4F6E3DC14BF0000E4C6E4D6E4E6E94
:1037F0004F5007E04B364B904C364D364E36FF0F50
:10380000F8D7900E4B264B0E4C22000E4D224BC08B
:10381000F6FF4CC0F7FF4DC0F8FF0900F5CF4EF1A1
:103820000900F5CF4FF10900F5CF50F10900F5CFB0
:1038300051F151514D5D08E150514C5D05E14F5141
:103840004B5D02E14E514A5D02E33D2BC6D789D064
:10385000010E3D6F3D51080A37E0020E4F6E3DC12B
:103860004BF0000E4C6E4D6E4E6E4F5007E04B36D7
:103870004B904C364D364E36FF0FF8D7B80E4B26D0
:103880004B0E4C22000E4D224BC0F6FF4CC0F7FFF2
:103890004DC0F8FF0900F5CF4EF10900F5CF4FF10B
:1038A0000900F5CF50F10900F5CF51F151514D5DAF
:1038B00008E150514C5D05E14F514B5D02E14E5125
:1038C0004A5D02E33D2BC6D74CD0010E3D6F3D5102
:1038D0000C0A37E0020E4F6E3DC14BF0000E4C6EED
:1038E0004D6E4E6E4F5007E04B364B904C364D367A
:1038F0004E36FF0FF8D7D80E4B264B0E4C22000E3B
:103900004D224BC0F6FF4CC0F7FF4DC0F8FF090039
:10391000F5CF4EF10900F5CF4FF10900F5CF50F189
:103920000900F5CF51F151514D5D08E150514C5D09
:1039300005E14F514B5D02E14E514A5D02E33D2BE3
:10394000C6D70FD05251000AD8B445D75251C00A39
:10395000D8B441D75251800AD8B47AD75251400ACC
:10396000B4E0800E4B6E800E3C194B5C02E13B5183
:103970003D5D03E23BC13DF10DD0800E3C194B6E25
:10398000800E4B5C02E13D513B5D04E23DC13BF1E9
:10399000000E3C6F3E513F110EE0030E40154B6E82
:1039A00041C14CF0000E4C164B504C1004E0010E7F
:1039B0003E5F000E3F5B800E3C194B6E800E3F1940
:1039C0004B5C02E13E513B5D05E23B513E5F3C51A9
:1039D0003F5B02D03E6B3F6BC40E40154E6F4151B2
:1039E000080B4F6F4F51080A02E1400E4E1908E1D3
:1039F0003E513F1104E0010E3E5F000E3F5B1CD0C4
:103A0000C00E40154E6F4151080B4F6F4F51080AC1
:103A100002E1800E4E1910E1800E4B6E800E3F19B0
:103A20004B5C02E13E51020805E2020E3E5F000ED1
:103A30003F5B02D03E6B3F6B40A56DD040A31AD0D8
:103A4000010E40154B6E41C14CF0000E4C164B5010
:103A50004C1003E02D0E4B6E02D02B0E4B6E2DC181
:103A6000E1FF2EC1E2FF4BC0E6FF2D4B2E2B424B58
:103A7000432B3CD0010E40154B6E41C14CF0000E63
:103A80004C164B504C100BE02DC1E1FF2EC1E2FF54
:103A9000200EE66E2D4B2E2B424B432B27D0C00E13
:103AA00040154E6F4151080B4F6F4F51080A02E10C
:103AB000800E4E191BE12DC1E1FF2EC1E2FF300E39
:103AC000E66E2D4B2E2B424B432B40AB03D0580EB2
:103AD0004B6E02D0780E4B6E2DC1E1FF2EC1E2FF7E
:103AE0004BC0E6FF2D4B2E2B424B432B3E513F113B
:103AF00011E02DC1E1FF2EC1E2FF300EE66E2D4B2D
:103B00002E2B424B432B010E3E5F000E3F5B3E517E
:103B10003F11EFE184D03E513F1113E040B711D087
:103B20002DC1E1FF2EC1E2FF200EE66E2D4B2E2BA4
:103B3000424B432B010E3E5F000E3F5B3E513F1157
:103B4000EFE140A31AD0010E40154B6E41C14CF07D
:103B5000000E4C164B504C1003E02D0E4B6E02D055
:103B60002B0E4B6E2DC1E1FF2EC1E2FF4BC0E6FFD5
:103B70002D4B2E2B424B432B14D0010E40154B6E78
:103B800041C14CF0000E4C164B504C100AE02DC1B8
:103B9000E1FF2EC1E2FF200EE66E2D4B2E2B424B95
:103BA000432BC00E40154E6F4151080B4F6F4F51C4
:103BB000080A02E1400E4E190BE12DC1E1FF2EC1B2
:103BC000E2FF300EE66E2D4B2E2B424B432B27D0BF
:103BD000C00E40154E6F4151080B4F6F4F51080AF0
:103BE00002E1800E4E191BE12DC1E1FF2EC1E2FF63
:103BF000300EE66E2D4B2E2B424B432B40AB03D0A9
:103C0000580E4B6E02D0780E4B6E2DC1E1FF2EC1C7
:103C1000E2FF4BC0E6FF2D4B2E2B424B432B800E79
:103C20004B6E800E3C194B5C02E13B513D5D0BE25B
:103C30002DC1E1FF2EC1E2FF300EE66E2D4B2E2B83
:103C4000424B432BECD73BC14BF03CC14CF0010E37
:103C50003B5F000E3C5B4B504C10D8B446D1C00EBD
:103C600040154B6E4BC04EF124D1020E4F6E3BC13E
:103C70004BF03CC14CF0000E3CBFFF0E4D6E4E6E43
:103C80004F5007E04B364B904C364D364E36FF0FBB
:103C9000F8D7900E4B264B0E4C22000E4D224BC0F7
:103CA000F6FF4CC0F7FF4DC0F8FF0900F5CF4FF00D
:103CB0000900F5CF50F00900F5CF51F00900F5CF1C
:103CC00052F04AC14BF04BC14CF04CC14DF04DC1CC
:103CD0004EF0F4EC0BF00A0E4F6E000E506E516E6B
:103CE000526EF4EC0BF053C04BF054C04CF055C086
:103CF0004DF056C04EF0300E4B2401013D6FE9D01F
:103D000040AB4CD0020E4F6E3BC14BF03CC14CF06F
:103D1000000E3CBFFF0E4D6E4E6E4F5007E04B360F
:103D20004B904C364D364E36FF0FF8D7B80E4B261B
:103D30004B0E4C22000E4D224BC0F6FF4CC0F7FF3D
:103D40004DC0F8FF0900F5CF4FF00900F5CF50F056
:103D50000900F5CF51F00900F5CF52F04AC14BF000
:103D60004BC14CF04CC14DF04DC14EF0F4EC0BF09A
:103D70000F0E4B16000E4C164D164E16080E4B2607
:103D80004C0E4C22000E4D224BC0F6FF4CC0F7FFEC
:103D90004DC0F8FF0900F5CF3DF14CD0020E4F6E3B
:103DA0003BC14BF03CC14CF0000E01013CBFFF0E8B
:103DB0004D6E4E6E4F5007E04B364B904C364D36A5
:103DC0004E36FF0FF8D7B80E4B264B0E4C22000E86
:103DD0004D224BC0F6FF4CC0F7FF4DC0F8FF090065
:103DE000F5CF4FF00900F5CF50F00900F5CF51F0B5
:103DF0000900F5CF52F04AC14BF04BC14CF04CC119
:103E00004DF04DC14EF0F4EC0BF00F0E4B16000EC2
:103E10004C164D164E161A0E4B264C0E4C22000E0A
:103E20004D224BC0F6FF4CC0F7FF4DC0F8FF090014
:103E3000F5CF3DF14ED0020E4F6E3BC14BF03CC171
:103E40004CF0000E01013CBFFF0E4D6E4E6E4F5008
:103E500007E04B364B904C364D364E36FF0FF8D7B9
:103E6000D80E4B264B0E4C22000E4D224BC0F6FFB7
:103E70004CC0F7FF4DC0F8FF0900F5CF4FF0090027
:103E8000F5CF50F00900F5CF51F00900F5CF52F011
:103E90004AC14BF04BC14CF04CC14DF04DC14EF0FE
:103EA000F4EC0BF0070E4B1401013D6F300E3D2773
:103EB00010D001014E51000AD8B4D7D64E51C00AD5
:103EC000D8B4D3D64E51800AD8B41AD74E51400A2E
:103ED000B2E02DC1E1FF2EC1E2FF3DC1E6FF0101CD
:103EE0002D4B2E2B424B432BAED6010140A71BD0AE
:103EF000800E4B6E800E3F194B5C02E13E51000874
:103F000012E22DC1E1FF2EC1E2FF200EE66E01019B
:103F10002D4B2E2B424B432B010E3E5F000E3F5B81
:103F20003E513F11EEE171EF0EF042C14BF043C143
:103F30004CF012000B6A2DC156F118EC0EF0010E78
:103F40000B6E120014D0800E01010C6F1ED0C00E3B
:103F500001010C6F1AD0940E01010C6F16D0D40E13
:103F600001010C6F12D0800E01010C6F0ED0010107
:103F70000C51010AE8E00C51020AE9E00C51030A75
:103F8000EAE00C51040AEBE0EED701010D054B6E9F
:103F90000C514B264BC00CF1010E0B6E4BC056F171
:103FA00018EC0EF00B6A0EC156F118EC0EF0010E73
:103FB0000B6E120001010D6B0E6B0F6B106B82907C
:103FC0000C6B200E01010C5D2AE20DC150F00EC1F8
:103FD00051F00FC152F010C153F05036509051368D
:103FE0005236533650C00DF151C00EF152C00FF190
:103FF00053C010F182844F6A82B24F2A4F50501042
:104000000D6F51C00EF152C00FF153C010F1000EF0
:104010000E130F131013829401010C2BD2D7828040
:10402000FF0E01010D15506EFF0E0E15516EFF0EA5
:104030000F15526E1F0E1015536E50C00DF151C06A
:104040000EF152C00FF153C010F1040E4F6E50C06C
:104050004BF051C04CF052C04DF053C04EF04F5099
:1040600009E04E324D324C324B324E9E4EBC4E8E9B
:10407000FF0FF6D74BC00DF14CC00EF14DC00FF144
:104080004EC010F112000001220E576E536A546A9E
:10409000556A566A5706D8B470EF20F0D890563259
:1040A0005532543253324E324D324C324B32D8A00C
:1040B0004AEF20F05706D8B468EF20F04F5053264F
:1040C0005050542251505522525056224FEF20F05A
:1040D0004F50532650505422515055225250562280
:1040E0001200110E01012B6F010E2C6F0CC12DF16E
:1040F0000DC12EF10EC12FF10FC130F110C131F100
:104100002B0E326F010E336F5FEC0EF04BC029F1B6
:104110004CC02AF14B5001010C25E16E4C500D2191
:10412000E26EE66A29C14BF02AC14CF0120001018F
:104130000E6B0F6B01010E510C25E96E0F510D2115
:10414000EA6EEECF4BF04B520EE00E510C25E96EAD
:104150000F510D21EA6EEECF2DF19AEC1FF0010107
:104160000E4B0F2BE7D712004C6AACB24C2A4C50C6
:10417000000A02E10000F8D70CC1ADFF1200010EE9
:104180000C184B6E4BC00CF04B520AE0010E0101B3
:104190000C6F140E0D6F2D0E0E6FA2EC1FF009D0D8
:1041A000010E01010C6F140E0D6F5F0E0E6FA2EC6D
:1041B0001FF0120011C00DF012C00EF013C00FF06E
:1041C00014C010F015C011F016C012F017C013F093
:1041D00018C014F019C015F01AC016F01BC017F063
:1041E0001CC018F01DC019F01EC01AF01FC01BF033
:1041F00020C01CF021C01DF022C01EF023C01FF003
:1042000024C020F025C021F026C022F027C023F0D2
:1042100028C024F029C025F02AC026F02BC027F0A2
:104220002CC028F02DC029F02EC02AF02FC02BF072
:1042300030C02CF031C02DF032C02EF033C02FF042
:1042400034C030F0DAEC1FF04BC031F04CC032F02B
:104250004DC033F04EC034F02D504B262E504C2222
:104260002F504D2230504E2229504B262A504C229E
:104270002B504D222C504E2225504B2626504C229E
:1042800027504D2228504E2221504B2622504C229E
:1042900023504D2224504E221D504B261E504C229E
:1042A0001F504D2220504E2219504B261A504C229E
:1042B0001B504D221C504E2215504B2616504C229E
:1042C00017504D2218504E2211504B2612504C229E
:1042D00013504D2214504E220D504B260E504C229E
:1042E0000F504D2210504E220A0E4F6E000E506E8F
:1042F000516E526EF4EC0BF0940E4F6E000E506E39
:10430000516E526E43EC20F0640E4F6E000E506EF4
:10431000516E526EF4EC0BF012004C6A9EBA4C2AAD
:104320004CC04BF01200AECF09F1ABA202D0AB985B
:10433000AB8809C14BF01200600E01010C6F000E3A
:104340000D6F2C0E0E6F4C0E0F6F000E106F35C0E0
:1043500011F136C012F137C013F138C014F107C0A3
:1043600015F108C016F105C017F106C018F171EC7F
:1043700020F0800E566F18EC0EF0600E01010C6FED
:10438000000E0D6F97EC20F0120001010B6B010184
:104390000B510925E96E000E0A21EA6EEECF4DF0B1
:1043A0004D50000A0DE00B510925E96E000E0A215F
:1043B000EA6EEECF0CF1B4EC20F001010B2BE7D745
:1043C00009C14BF00AC14CF01200A69CFDC0A9FF28
:1043D000A69EA680A8CF4BF01200FDC009F0FEC03B
:1043E0000AF0FDC0E1FFFEC0E2FFE66AFDC009F091
:1043F000FEC00AF0110EE126E76A120EE15EE2EC61
:1044000004F0E78AE788E786E0EC04F0E796E2EC60
:1044100004F0E78AE788E786E0EC04F0E796F1EC41
:1044200004F0F1EC04F0E78AE788E786E0EC04F0BA
:10443000E796E2EC04F0E78AE798E786E0EC04F020
:10444000E796F1EC04F0E78AE798E786E0EC04F001
:10445000E796E78EE79CE786E0EC04F0E796F1EC60
:1044600004F0000EE76EE786E0EC04F0E796E78ED6
:10447000E78CE78AE788E786E0EC04F0E796F1EC62
:1044800004F0000EE76EE786E0EC04F0E796E788BC
:10449000E786E0EC04F0E796E2EC04F0000EE76E4D
:1044A000E786E0EC04F0E796E78CE78AE786E0EC45
:1044B00004F0E796F1EC04F0010E0B6E12000C0E06
:1044C0000101566F18EC0EF0010E00144B6ED8B4BB
:1044D00039D10090BFEC20F0DAEC20F0DBEC0BF0EF
:1044E000950E4F6EBF0E506E560E516E670E526E89
:1044F000E1EC01F039C04FF03AC050F03BC051F050
:104500003CC052F0EFEC0BF04BC0FDF04CC0FEF0A5
:104510004DC0FFF04EC000F1FDC03DF0FEC03EF0CA
:10452000FFC03FF000C140F0FDC04BF0FEC04CF0BA
:10453000FFC04DF000C14EF0000E4F6E240E506EC5
:10454000740E516E920E526EE1EC01F0E10E4F6E60
:104550007A0E506E240E516E810E526E94EC0AF05B
:104560004BC0F9F04CC0FAF04DC0FBF04EC0FCF06F
:104570004BC041F04CC042F04DC043F04EC044F03F
:10458000600E01010C6F000E0D6F400E0E6F4C0E91
:104590000F6F000E106FFDC011F1FEC012F1FFC0D1
:1045A00013F100C114F14BC015F14CC016F14DC010
:1045B00017F14EC018F171EC20F0C00E566F18ECD8
:1045C0000EF0600E01010C6F000E0D6F97EC20F0E5
:1045D000000E4F6E000E506E7A0E516E880E526EA7
:1045E000F9C04BF0FAC04CF0FBC04DF0FCC04EF0EF
:1045F000AFEC09F0010ED8B0000E4B6E4B52D8B4A0
:10460000A1D04F6A506A516A526AF9C04BF0FAC0A1
:104610004CF0FBC04DF0FCC04EF0AFEC09F0000ECA
:10462000D8B0010E4B6E4B52D8B48CD045C04BF075
:1046300046C04CF047C04DF048C04EF0F9C04FF0B6
:10464000FAC050F0FBC051F0FCC052F0CCEC02F0CC
:104650004BC045F04CC046F04DC047F04EC048F04E
:10466000F9C04FF0FAC050F0FBC051F0FCC052F05E
:10467000E0C04BF0E1C04CF0E2C04DF0E3C04EF0C2
:10468000AFEC09F0010ED8B0000E4B6E4B5228E093
:10469000F9C0E0F0FAC0E1F0FBC0E2F0FCC0E3F0EA
:1046A000600E01010C6F000E0D6F520E0E6F4C0E5E
:1046B0000F6F000E106FF9C011F1FAC012F1FBC0BC
:1046C00013F1FCC014F171EC20F0D40E566F18EC0D
:1046D0000EF0600E01010C6F000E0D6F97EC20F0D4
:1046E000600E01010C6F000E0D6F620E0E6F4C0E0E
:1046F0000F6F000E106F000E4F6E000E506E610EA9
:10470000516E8A0E526E45C04BF046C04CF047C009
:104710004DF048C04EF094EC0AF04BC011F14CC083
:1047200012F14DC013F14EC014F171EC20F0940E53
:10473000566F18EC0EF0600E01010C6F000E0D6F3D
:1047400097EC20F01200000E081802E1140E071872
:1047500017E1000E061802E1000E051811E1000E27
:10476000041802E1000E03180BE1376A386A456A43
:10477000466A476A486A0001E06BE16BE26BE36BF3
:1047800012008DEC21F04B5205E093EC21F04BC070
:1047900049F002D0FF0E496E12004950680A0AE043
:1047A000010E80144C6E4C50000A03E14A50000A7E
:1047B00001E011D0010E4A6E074A082A800E08183F
:1047C0004B6E800E4B5C02E1180E075C02E3076A39
:1047D000086A9CEC21F080B04A6A120049506D0AC8
:1047E0000CE04C6A80B44C2A4C50000A04E10001F1
:1047F000E451000A02E0000114D0010E0001E46F50
:10480000036A046A054A062A800E4B6E800E06185B
:104810004B5C02E105503B0802E2056A066A9CEC2B
:1048200021F080A402D00001E46B120049507A0A02
:1048300016E1DAEC20F0DBEC0BF0950E4F6EBF0EBC
:10484000506E560E516E670E526EE1EC01F04BC089
:1048500039F04CC03AF04DC03BF04EC03CF0120075
:1048600000A280D00092374A382A600E01010C6FF6
:10487000000E0D6F740E0E6F4C0E0F6F000E106F4A
:1048800035C011F136C012F137C013F138C014F140
:1048900007C015F108C016F105C017F106C018F1E0
:1048A00071EC20F0800E566F18EC0EF0600E0101D6
:1048B0000C6F000E0D6F97EC20F0600E01010C6F75
:1048C000000E0D6F880E0E6F4C0E0F6F000E106FE6
:1048D00035C011F136C012F137C013F138C014F1F0
:1048E00007C015F108C016F105C017F106C018F190
:1048F0003DC019F13EC01AF13FC01BF140C01CF190
:1049000041C01DF142C01EF143C01FF144C020F15F
:10491000E0C021F1E1C022F1E2C023F1E3C024F1C3
:10492000000E4F6E000E506E610E516E8A0E526E6A
:1049300045C04BF046C04CF047C04DF048C04EF06B
:1049400094EC0AF04BC025F14CC026F14DC027F184
:104950004EC028F171EC20F0600E096F000E0A6F56
:10496000C5EC21F01200530E0001E56F4F0EE66F0B
:104970004C0EE76F410EE86F520EE96F200EEA6FA2
:10498000530EEB6F540EEC6F410EED6F540EEE6F45
:10499000490EEF6F4F0EF06F4E0EF16F200EF26F5B
:1049A000300EF36F310EF46FF56BE50EF66F000EFF
:1049B000F76F000E376E000E386E000EF86F000EA7
:1049C000016E000E026E000E036E000E046E000EED
:1049D000006E000E396E000E3A6E000E3B6E000E39
:1049E0003C6E000E456E000E466E000E476E000EC9
:1049F000486E000E4A6E000EE46F000E0C6E000E44
:104A0000E06F000EE16F000EE26F000EE36F120028
:104A1000AC8A900EAB6E948E949C9EAA03D0AECFBF
:104A2000FDF0FBD71200B3EC24F0020E576EFF0E20
:104A3000566EFF0E556E572E01D007D0562E01D060
:104A400003D0552EFED7FAD7F6D7870E566EFF0E37
:104A5000556E562E01D003D0552EFED7FAD7930EA1
:104A6000556E552EFED700000F0EC16EEF0E926EE2
:104A7000936AFF0E826E820E946E020E576EFF0EC8
:104A8000566EFF0E556E572E01D007D0562E01D010
:104A900003D0552EFED7FAD7F6D7060E566EFF0E68
:104AA000556E562E01D003D0552EFED7FAD70A0EDA
:104AB000556E552EFED7310ECD6E010E9D6EC00E79
:104AC000F26E829E080E076E000E086E056A066A78
:104AD000190EAF6EAC8408EC25F00001FD6BE5EC1F
:104AE00021F04BC035F0000E366E810E0001FD6FD7
:104AF0000F0EFE6FEDEC21F00001E06BE16BE26B5D
:104B0000E36B006A9CEC21F05FEC22F0A3EC23F055
:104B1000C1EC23F0CDEC23F0EEEC23F016EC24F006
:104B200030EC24F0F1D7FFD70000007FCDCC4C7BD8
:104B30000AD723786F12037517B75171ACC5276E6A
:104B4000BD37066B95BF566777CC2B645F700961E4
:104B5000FFE65B5D08E53C3C6042221B0000007FF5
:104B6000000020820000488500007A8800401C8CEC
:104B70000050438F002474928096189620BC3E9972
:104B8000286B6E9CF90215A0EC782DC1CAF249E29F
:104B9000010000000A00000064000000E8030000BB
:104BA00010270000A086010040420F008096980068
:104BB00000E1F50500CA9A3B01000000100000006A
:104BC00000010000001000000000010000001000C3
:104BD00000000001000000100100000008000000BB
:104BE00040000000000200000010000000800000F3
:104BF0000000040000002000000000010000000888
:104C000000000040000000003031323334353637C8
:104C1000383941424344454600FF30313233343560
:104C20003637383961626364656600FF2530336466
:104C30002C253035642C253032643A25303264001E
:104C4000454D463D25302E3666562025302E3166A0
:104C500000FF4D41583D25302E316620572F6D5EA7
:104C6000320073756D3D25302E30662057482F6D0C
:104C70005E3200FF253033642C253035642C25301E
:104C800032643A25303264000A25642C25642C25D0
:104C90003032643A253032642C25302E36662C258D
:104CA000302E31662C25302E31662C25302E306684
:104CB00000FFFFFFFFFFFFFFFFFFFFFFFFFFFFFF03
:020000040030CA
:0E000000FFF8FFFEFFFFBBFFFFFFFFFFFFFF4C
:00000001FF
